:100000000C94280018950000189500001895000021
:10001000189500001895000018950000189500002C
:10002000189500000C94120D18950000189500000A
:10003000189500001895000018950000189500000C
:1000400018950000189500001895000018950000FC
:100050008FE181BD87E181BD8FE58DBFC4E0E8E719
:100060004E2E88E08EBFD8E0F7E05F2EEEEFF7E08F
:10007000A0E6B0E088278D933197E9F783E389B94B
:1000800088E18AB9662481E48ABB81E38BBB8FEB6C
:1000900087BB8FEB88BB88E084BB83E085BB80E0B7
:1000A00081BB8BE382BB80E08FBD81E08EBD8FE1A1
:1000B00081BD87E181BD86E086B980E487B9C398B8
:1000C000C29AD89ADE9AC498C798C598F894A89509
:1000D0007091D100777F7093D1007091D1007B7FB8
:1000E0007093D1000027A1EDB0E08C9183FB0EF45A
:1000F00001E041E0041781E009F080E08F930027E0
:10010000A1EDB0E08C9182FB0EF401E041E0041718
:1001100081E009F080E09F91892B882311F40C94F1
:100120009400DC9881E58ABB0E94810E7091D10019
:1001300070627093D100EFEFF1E0A2ECB0E091E0DB
:100140000E949F2F0091C200003081E009F080E002
:100150008F930091C2000E3F80E010F009F081E023
:100160009F91892B882311F40C94B9008EEB809316
:10017000C2000091C2004AE0040F01BF89E190E093
:100180000E94912EE4E9FFE50E94D82D0027A1ED01
:10019000B0E08C9183FB0EF401E041E0041711F014
:1001A0000C94DA00EEEAFFE50E94D82D0E94E42DBF
:1001B0000C94ED00E0EBFFE50E94D82DA1EDB0E03E
:1001C0008C9182FBA8E6B7E00E94B62E8D9388271B
:1001D0008C930E94D02D0E94E42DEAE0F0E0BB2732
:1001E000A0E10E949C2F073411F40C942D01EBE048
:1001F000F0E0A0E1BB278FE08C937BE70E948B2F80
:10020000ECE0F0E001E010E0A0E1BB277BE70E941A
:100210008D2FEAE0F0E0A0E1BB2787E48C937BE739
:100220000E948B2FEEE0F0E0A0E1BB2780E08C93F2
:100230007BE70E948B2FE0E1F0E000E010E0A0E11E
:10024000BB277BE70E948D2FEFE0F0E0A0E1BB270A
:1002500080E08C937BE70E948B2FEBE0F0E0ABEB30
:10026000B0E00E949C2F0091BB00043618F011F002
:100270000C943C010C943F0184E68093BB0080E722
:1002800097E9ACEBB0E08D939C93ECE0F0E0A6EB4B
:10029000B0E00E949E2FEEE0F0E0A3ECB0E00E9400
:1002A0009C2FEFE0F0E0A4ECB0E00E949C2F0E94B5
:1002B000850EE0E1F0E0A3E6B0E00E949E2FA3E609
:1002C000B0E00E943F2DE0E1F0E0A3E6B0E07BE784
:1002D0000E948D2FA6EBB0E00D911C91003050E0F4
:1002E000150711F00C947A0181E090E0A6EBB0E0E4
:1002F0008D939C93E2EBFFE50E94D82DA8E6B7E032
:10030000EBEBF0E00E94242F0E94D02DEAEBFFE5FA
:100310000E94D82DA8E6B7E0E6EBF0E00E94152F8A
:100320000E94D02DEAEBFFE50E94D82DA8E6B7E0A9
:10033000E3ECF0E00E94242F0E94D02DEAEBFFE5D1
:100340000E94D82DA8E6B7E0E4ECF0E00E94242F4C
:100350000E94D02DEAEBFFE50E94D82DA8E6B7E079
:10036000E3E6F0E00E94152F0E94D02D0E94E42DBC
:1003700080E08093D00070916A00777F70936A006C
:1003800080E08093C60086E08093BE008DE080937D
:10039000BF00E9E6F0E0FA93EA930E94D71D2296A7
:1003A00084E190E00E94912EDE980E947D2EC49AF6
:1003B000ECEBFFE50E94D82D0E94E42D88EC90E044
:1003C0000E94912EA89581B5886181BD877F81BDEE
:1003D000E0E6F0E0FA93EA930E944D222296A89577
:1003E00000916000003011F40C9402020E9461211F
:1003F000E6ECFFE50E94D82D0E94E42D0E94480EF5
:100400000C9407027091D1007F7B7093D100E0EDD6
:10041000FFE50E94D82D0E948A2184E690E00E9488
:10042000912E00916900003018F011F00C941A021E
:100430000C942102E9E6F0E0FA93EA930E94661F29
:1004400022960027A1EDB0E08C9186FB0EF401E02E
:1004500040E0041711F00C942F020E9414158FEF46
:100460000E94E72D82E390E00E94912E7894A89557
:1004700081B5886081BDA2EBB0E04D915C91A6EBA7
:10048000B0E00D911C910417150718F011F00C94B1
:100490004B020C94510281E090E0A6EBB0E08D930A
:1004A0009C930027AAE6B0E08C9184FB0EF401E057
:1004B00041E0041781E009F080E08F930027A1ED6F
:1004C000B0E08C9186FB0EF401E040E0041781E07F
:1004D00009F080E09F918923882311F40C94830212
:1004E000E6EBF0E0FA93EA935A924A9280E0A42D68
:1004F000B52D8C9381E00E942C2D0E94C21224966F
:1005000081E00E94282D80E08093B80080E08093F5
:10051000690070916A007F7770936A000027A1EDEF
:10052000B0E08C9186FB0EF401E041E0041711F07D
:100530000C949C020E94810EA895ABE6B0E088273F
:100540008C930027A1EDB0E08C9183FB0EF401E0C9
:1005500041E0041711F00C94B4020E94C82DABE6E0
:10056000B0E08D9388278C93ABE6B0E08C9180301F
:1005700011F00C9487050091D000003081E009F063
:1005800080E08F930027AAE6B0E08C9181FB0EF407
:1005900001E040E0041781E009F080E09F91892BA1
:1005A000882311F40C945704E0E6F0E0FA93EA9300
:1005B0000E942F1E229600916000003018F011F06A
:1005C0000C94E4020C94570470916A007068709364
:1005D0006A000091D200003011F00C944003409169
:1005E000C60000916000041718F011F00C94FA0294
:1005F0000C944003809160008093C6000027AAE617
:10060000B0E08C9184FB0EF401E040E0041711F09F
:100610000C941A03A0E6B0E08C91A6EBB0E08D93A9
:1006200088278C93ABE6B0E0EAEDFFE50E94B72D9A
:100630000C9440030027A1EDB0E08C9187FB0EF4F1
:1006400001E041E0041711F00C943A03A0E6B0E099
:100650000D91112741E050E0040F151FA6EBB0E00B
:100660000D931C93ABE6B0E0EAEDFFE50E94B72DD9
:100670000C944003ABE6B0E0ECEDFFE50E94B72D33
:100680000091D200013011F00C94D403009160006D
:10069000013011F00C945203ABE6B0E0ECEDFFE555
:1006A0000E94B72D00916000023011F00C945E039F
:1006B000ABE6B0E0EEEDFFE50E94B72D80E0809361
:1006C000620000916000033081E009F080E08F93C8
:1006D0000091BB00043681E008F080E09F918923FF
:1006E000882311F40C947C03ABEBB0E08C918E5F0B
:1006F0008C9381E08093620000916000043081E07F
:1007000009F080E08F930091BB00023080E010F090
:1007100009F081E09F918923882311F40C949803B8
:10072000ABEBB0E08C9182508C9381E080936200BF
:1007300000916200013011F00C94D4038EB5887FD3
:100740008EBD5A924A928091BB00A42DB52D8C93F8
:1007500081E00E942C2D5A924A928091C000A42DD3
:10076000B52D8C9381E00E942C2D5A924A92809153
:10077000C100A42DB52D8C9381E00E942C2D0E94E8
:100780003B29269683E00E94282DEBE0F0E0ABEBBE
:10079000B0E07BE70E948B2F0091D000013011F078
:1007A0000C94D40381E08EBD0091D200023011F090
:1007B0000C9457044091C60000916000041718F093
:1007C00011F00C94E5030C94570480916000809321
:1007D000C60000916000013011F00C94FB0381E031
:1007E00090E0A6EBB0E08D939C93ABE6B0E0EAED31
:1007F000FFE50E94B72D00916000023011F00C94CB
:100800003F04A2EBB0E00D911C9141E050E0041BCD
:10081000150BA3E6B0E00D931C9302E010E00F93DC
:100820001F93A3E6B0E08D919C918A939A930E94C6
:10083000582D2296402F512F1F910F91040F151FF5
:10084000A3E6B0E00D931C93A6EBB0E04D915C9154
:10085000A3E6B0E00D911C910417150711F40C9458
:100860000104A3E6B0E08D919C91A6EBB0E08D93DE
:100870009C93ABE6B0E0EAEDFFE50E94B72D009156
:100880006000033011F00C944B04ABE6B0E0ECEDEB
:10089000FFE50E94B72D00916000043011F00C9428
:1008A0005704ABE6B0E0EEEDFFE50E94B72D002760
:1008B000AAE6B0E08C9184FB0EF401E041E004175D
:1008C00081E009F080E08F930027A1EDB0E08C91EA
:1008D00087FB0EF401E041E0041781E009F080E0BD
:1008E0009F9189238F930091D000013081E009F01E
:1008F00080E09F918923882311F40C94C204A6EB15
:10090000B0E00D911C91013050E0150711F00C94EE
:10091000C204E0E6F0E0FA93EA930E942F1E2296CA
:1009200000916000003080E010F009F081E08F93CA
:10093000A2EBB0E04D915C91A0E6B0E00D911127E3
:100940000417150781E008F080E09F918923882330
:1009500011F40C94C204A0E6B0E00D91112741E01F
:1009600050E0040F151FA6EBB0E00D931C93ABE60F
:10097000B0E0EAEDFFE50E94B72D70916A00706863
:1009800070936A000027AAE6B0E08C9180FB0EF419
:1009900001E040E0041711F00C948705E9E6F0E06F
:1009A000FA93EA930E94D71D2296009169000430C1
:1009B00011F00C94E2040E94190E70916A007068A4
:1009C00070936A0080E080936000009169000230BB
:1009D00081E009F080E08F930091BB00043681E054
:1009E00008F080E09F918923882311F40C9400057E
:1009F000ABEBB0E08C918B5F8C9381E080936000D7
:100A000000916900033081E009F080E08F9300914C
:100A1000BB00053081E009F080E09F9189238823A5
:100A200011F40C94190581E08093BB0081E0809360
:100A3000600000916900033081E009F080E08F934D
:100A40000091BB00053080E010F009F081E09F913B
:100A50008923882311F40C943505ABEBB0E08C911D
:100A600085508C9381E0809360000091600001309C
:100A700011F00C9476058EB5887F8EBD5A924A92FD
:100A80008091BB00A42DB52D8C9381E00E942C2D6C
:100A90005A924A928091C000A42DB52D8C9381E08A
:100AA0000E942C2D5A924A928091C100A42DB52DFE
:100AB0008C9381E00E942C2D0E943B29269683E096
:100AC0000E94282DEBE0F0E0ABEBB0E07BE70E946A
:100AD0008B2F0091D000013011F00C94710581E052
:100AE0008EBD70916A00706870936A000091690011
:100AF000013011F00C948705ABE6B0E0ECEDFFE5BA
:100B00000E94B72D70916A00706870936A00EBE6DE
:100B1000F0E0ABE6B0E00E94AA2EABE6B0E08C912C
:100B2000803081E009F480E08F930091690000300B
:100B300081E009F480E09F91892B8F930091B800A8
:100B4000013081E009F080E09F91892B882311F426
:100B50000C948E020091B800013011F00C94D10574
:100B600080E08093B800ABE6B0E0ECEDFFE50E94DA
:100B7000B72D0027A1EDB0E08C9187FB0EF401E0CA
:100B800041E0041711F00C94D10581E090E0A6EB50
:100B9000B0E08D939C93ABE6B0E0EAEDFFE50E94F8
:100BA000B72DABE6B0E0E0EEFFE50E94B62F11F006
:100BB0000C941B060E94C42DA0E6B0E08C9300911B
:100BC0006000003011F40C94DA050E94C82DA0ECEE
:100BD000B0E08C938EB5887F8EBD5A924A928091F8
:100BE000BB00A42DB52D8C9381E00E942C2D5A9230
:100BF0004A928091C000A42DB52D8C9381E00E9473
:100C00002C2D5A924A928091C100A42DB52D8C931F
:100C100081E00E942C2D0E943B29269683E00E94B1
:100C2000282D0091D000013011F00C94190681E0BC
:100C30008EBD0C94440CE2EEFFE50E94B62F11F03D
:100C40000C9463060E94C42DA0E6B0E08C93009142
:100C50006000003011F40C9422060E94C82DA1EC13
:100C6000B0E08C938EB5887F8EBD5A924A92809167
:100C7000BB00A42DB52D8C9381E00E942C2D5A929F
:100C80004A928091C000A42DB52D8C9381E00E94E2
:100C90002C2D5A924A928091C100A42DB52D8C938F
:100CA00081E00E942C2D0E943B29269683E00E9421
:100CB000282D0091D000013011F00C94610681E0E4
:100CC0008EBD0C94440CE4EEFFE50E94B62F11F0AB
:100CD0000C94A8065A924A928091BE00A42DB52D7C
:100CE0008C9381E00E942C2D5A924A928091BF00F1
:100CF000A42DB52D8C9381E00E942C2D0E94032AF7
:100D0000249682E00E94282D0091C40041E0042B2B
:100D1000A0E6B0E00C937091D10070617093D100A7
:100D20008EB5887F8EBDEFE0F0E0A0E6B0E07BE717
:100D30000E948B2F809160008093C4000091D000AE
:100D4000013011F00C94A60681E08EBD0C94440C89
:100D5000E6EEFFE50E94B62F11F00C94EB065A92D6
:100D60004A9280E0A42DB52D8C9381E00E942C2D19
:100D70005A924A9280E0A42DB52D8C9381E00E9476
:100D80002C2D0E94032A249682E00E94282D009197
:100D9000C4004EEF0423A0E6B0E00C937091D100A4
:100DA0007F7E7093D1008EB5887F8EBDEFE0F0E03E
:100DB000A0E6B0E07BE70E948B2F809160008093DB
:100DC000C4000091D000013011F00C94E90681E0DC
:100DD0008EBD0C94440CEAEDFFE50E94B62F11F095
:100DE0000C945B070091D000013011F00C94FA06CE
:100DF0000E94190EA2EBB0E04D915C91A6EBB0E021
:100E00000D911C910417150718F011F00C9456075A
:100E10000027A1EDB0E08C9186FB0EF401E040E0EC
:100E2000041711F00C942707E6EBF0E0FA93EA932D
:100E30005A924A9280E0A42DB52D8C9381E00E94B5
:100E40002C2D0E94C212249681E00E94282D00279A
:100E5000A1EDB0E08C9186FB0EF401E041E00417B7
:100E600011F00C9454070E94480E0027A1EDB0E049
:100E70008C9186FB0EF401E040E0041711F00C9415
:100E80005407E6EBF0E0FA93EA935A924A9280E034
:100E9000A42DB52D8C9381E00E942C2D0E94C212AE
:100EA000249681E00E94282D0C94590780E08093BD
:100EB000C6000C94440CE8EEFFE50E94B62F11F03A
:100EC0000C9469070E94190E80E08093C6000C9470
:100ED000440CEAEEFFE50E94B62F11F00C94A30734
:100EE0000091D000013011F00C94A1070027AAE670
:100EF000B0E08C9183FB0EF401E040E0041711F0A8
:100F00000C9493078EB5887F8EBD89B78B7F89BF80
:100F100070916A00786070936A0084E690E00E94A5
:100F2000912E0C94A10770916A00777F70936A00EC
:100F300080E29EE49DBD8CBD81E08EBD89B784605A
:100F400089BF0C94440CECEDFFE50E94B62F11F024
:100F50000C943B080091D000013011F00C94B207C2
:100F60000E94190EA6EBB0E00E943F2D0027A1EDD4
:100F7000B0E08C9185FB0EF401E041E0041711F024
:100F80000C94D7070027AAE6B0E08C9184FB0EF4FE
:100F900001E040E0041711F00C94D207A6EBB0E09A
:100FA0000E94452D7091D1007F7D7093D100A2EBFE
:100FB000B0E04D915C91A6EBB0E00D911C9104174F
:100FC000150718F011F00C94E7070C94ED0781E079
:100FD00090E0A6EBB0E08D939C930027A1EDB0E0EC
:100FE0008C9186FB0EF401E040E0041711F00C94A4
:100FF0000C08E6EBF0E0FA93EA935A924A9280E00A
:10100000A42DB52D8C9381E00E942C2D0E94C2123C
:10101000249681E00E94282D0027A1EDB0E08C915C
:1010200086FB0EF401E041E0041711F00C9439083E
:101030000E94480E0027A1EDB0E08C9186FB0EF4D3
:1010400001E040E0041711F00C943908E6EBF0E001
:10105000FA93EA935A924A9280E0A42DB52D8C938C
:1010600081E00E942C2D0E94C212249681E00E94F1
:10107000282D0C94440CEEEDFFE50E94B62F11F0E4
:101080000C94B3080091D000013011F00C944A0880
:101090000E94190EA6EBB0E00D911C91013050E0BA
:1010A000150718F011F00C9457080C945D08A6EB86
:1010B000B0E00E94452D0C946508A2EBB0E08D9144
:1010C0009C91A6EBB0E08D939C930027A1EDB0E03E
:1010D0008C9186FB0EF401E040E0041711F00C94B3
:1010E0008408E6EBF0E0FA93EA935A924A9280E0A1
:1010F000A42DB52D8C9381E00E942C2D0E94C2124C
:10110000249681E00E94282D0027A1EDB0E08C916B
:1011100086FB0EF401E041E0041711F00C94B108D5
:101120000E94480E0027A1EDB0E08C9186FB0EF4E2
:1011300001E040E0041711F00C94B108E6EBF0E098
:10114000FA93EA935A924A9280E0A42DB52D8C939B
:1011500081E00E942C2D0E94C212249681E00E9400
:10116000282D0C94440CECEEFFE50E94B62F11F0F4
:101170000C942609A6EBB0E00E943F2DA2EBB0E054
:101180004D915C91A6EBB0E00D911C9104171507F1
:1011900018F011F00C94CE080C94D40881E090E083
:1011A000A6EBB0E08D939C938EB5887F8EBDA2E7B1
:1011B000B0E00D911D912D913C91A2E9B0E00D930D
:1011C0001D932D933C930027A1EDB0E08C9186FBFD
:1011D0000EF401E040E0041711F00C941C095A923F
:1011E0004A92A2E9B0E00D911D912D913C91A42D60
:1011F000B52D0D931D932D933C9384E00E942C2DCF
:101200005A924A92A6EBB0E08D919C91A42DB52DF7
:101210008D939C9382E00E942C2D5A924A9280E0FA
:10122000A42DB52D8C9381E00E942C2D0E942316B5
:10123000269687E00E94282D0091D000013011F001
:101240000C94240981E08EBD0C94440CE0EBFFE586
:101250000E94B62F11F00C949A09A6EBB0E00D9104
:101260001C91013050E0150718F011F00C943A0968
:101270000C944009A6EBB0E00E94452D0C9448095F
:10128000A2EBB0E08D919C91A6EBB0E08D939C9386
:101290008EB5887F8EBDA2E7B0E00D911D912D9196
:1012A0003C91A2E9B0E00D931D932D933C93002750
:1012B000A1EDB0E08C9186FB0EF401E040E0041754
:1012C00011F00C9490095A924A92A2E9B0E00D9163
:1012D0001D912D913C91A42DB52D0D931D932D9312
:1012E0003C9384E00E942C2D5A924A92A6EBB0E0E7
:1012F0008D919C91A42DB52D8D939C9382E00E949D
:101300002C2D5A924A9280E0A42DB52D8C9381E029
:101310000E942C2D0E942316269687E00E94282DDD
:101320000091D000013011F00C94980981E08EBD3D
:101330000C94440CEEEEFFE50E94B62F11F00C94D5
:10134000AA09ECE0F0E0A6EBB0E07BE70E948D2F6D
:101350000C94440CE0EFFFE50E94B62F11F00C94C2
:10136000BE098DE181BD85E181BD0E94190E81B567
:10137000886081BD0C94BA090C94440CABE6B0E0D3
:10138000E2EFFFE50E94B62F81E008F480E08F9342
:10139000ABE6B0E0E4EFFFE50E94B62F81E010F08D
:1013A00009F080E09F918923882311F40C94920A1C
:1013B00089B78B7F89BF8EB5887F8EBD0E94C42D73
:1013C000A0E6B0E08C9300916000003011F40C9422
:1013D000DE090E94C82DA6EBB0E08D9388278C9380
:1013E00080E08093D00070916A00777F70936A00EC
:1013F000A2EBB0E04D915C91A6EBB0E00D911C9199
:101400000417150780E010F009F081E08F93A6EB38
:10141000B0E00D911C91003050E0150781E009F01B
:1014200080E09F91892B882311F40C94320A81E08B
:1014300090E0A6EBB0E08D939C93E6EBF0E0FA939E
:10144000EA935A924A9281E0A42DB52D8C9381E0C3
:101450000E942C2D0E94C212249681E00E94282D09
:101460000C94900A0027A1EDB0E08C9186FB0EF45D
:1014700001E040E0041781E009F080E08F93ABE6E3
:10148000B0E0E2EFFFE50E94B62F81E009F080E0D6
:101490009F918923882311F40C94610AE6EBF0E014
:1014A000FA93EA935A924A9281E0A42DB52D8C9337
:1014B00081E00E942C2D0E94C212249681E00E949D
:1014C000282D0027A1EDB0E08C9186FB0EF401E001
:1014D00040E0041781E009F080E08F93ABE6B0E0D4
:1014E000E4EFFFE50E94B62F81E009F080E09F91D4
:1014F0008923882311F40C94900AE6EBF0E0FA9328
:10150000EA935A924A9280E0A42DB52D8C9381E003
:101510000E942C2D0E94C212249681E00E94282D48
:101520000C94440CE6EFFFE50E94B62F11F00C94EA
:10153000E10A0E94C42DA0E6B0E08C930091600007
:10154000003011F40C94990A0E94C82DABEBB0E066
:101550008C938EB5887F8EBD5A924A928091BB0043
:10156000A42DB52D8C9381E00E942C2D5A924A9285
:101570008091C000A42DB52D8C9381E00E942C2D6C
:101580005A924A928091C100A42DB52D8C9381E08E
:101590000E942C2D0E943B29269683E00E94282D34
:1015A000EBE0F0E0ABEBB0E07BE70E948B2F00912B
:1015B000D000013011F00C94DF0A81E08EBD0C9454
:1015C000440CE8EFFFE50E94B62F11F00C942F0BAE
:1015D0000E94C42DA0E6B0E08C9300916000003022
:1015E00011F40C94E80A8091C300809360000E947B
:1015F000C82DA3ECB0E08C93A3ECB0E08C918F737A
:101600008C930E94850E0091C30040E10423A0E664
:10161000B0E00C9300916000003111F00C94140BB9
:101620000E94810E0C94160B0E94830EA3ECB0E076
:101630008C918F7E8C938EB5887F8EBDEEE0F0E02E
:10164000A3ECB0E07BE70E948B2F0091D00001302B
:1016500011F00C942D0B81E08EBD0C94440CEEEA3D
:10166000FFE50E94B62F11F00C94930B0091C3007C
:101670004FE30423A0E6B0E00C930091D0000130CA
:1016800011F00C94480BA0E6B0E08C9180588C933C
:101690000027A1EDB0E08C9186FB0EF401E041E063
:1016A000041711F00C94590BA0E6B0E08C91805C0B
:1016B0008C930027AAE6B0E08C9183FB0EF401E046
:1016C00041E0041711F00C946A0BA0E6B0E08C9195
:1016D000805E8C938091B600809362008EB5887F87
:1016E0008EBD31E0A0E6B0E00E94DF2D31E0ABEB33
:1016F000B0E00E94DF2D31E0A2E6B0E00E94DF2DD5
:101700008091B2008093620031E0A2E6B0E00E94D6
:10171000DF2D0091D000013011F00C94910B81E08D
:101720008EBD0C94440CEAEFFFE50E94B62F11F039
:101730000C94160CA7EDB0E00D911D912D913C91EC
:10174000A3EDB0E04D915D916D917C910E94FD2ED5
:10175000A5E6B0E00D931D932D933D93A5E6B0E073
:101760000E94302DA5E6B0E00D911D912D913C9188
:1017700040E052E060E070E00E94F12DA5E6B0E0AC
:101780000D931D932D933D93A5E6B0E00D911D9112
:101790002D913C91A5ECB0E04C9155276627772719
:1017A0000E94F62DA5E6B0E04D935D936D937D9379
:1017B000A5E6B0E00D911D912D913C914AE050E0DD
:1017C00060E070E00E94F62DA5E6B0E04D935D93D9
:1017D0006D937D9344E150E060E070E0A5E6B0E0F9
:1017E0000D911D912D913C910E94022F0CF402C08D
:1017F0000C94040C00E010E020E030E0A5E6B0E03E
:101800000D931D932D933C938EB5887F8EBD34E050
:10181000A5E6B0E00E94DF2D0091D000013011F06C
:101820000C94140C81E08EBD0C94440CECEFFFE59D
:101830000E94B62F11F00C942E0C8EB5887F8EBDB1
:10184000A4EAB0E00E94D22D0091D000013011F046
:101850000C942C0C81E08EBD0C94440CEEEFFFE553
:101860000E94B62F11F00C94440C8EB5887F8EBD6B
:101870000E94BF150091D000013011F00C94420C71
:1018800081E08EBD0C94440C81E090E00E94912E8A
:101890000027AAE6B0E08C9187FB0EF401E040E05F
:1018A000041718F011F00C94570C0C94100D0091C3
:1018B0006900003018F011F00C94600C0C94C70C07
:1018C000A895E0E6F0E0FA93EA930E94D71D2296ED
:1018D00000916000043011F00C94BB0C0E94190EB2
:1018E00080E08093C6000E94830E85E090E00E9415
:1018F000912E80E080936200E0E6F0E0FA93EA93B4
:101900000E94D71D2296A2E6B0E08C918F5F8C9347
:1019100088E090E00E94912E00916000003081E00C
:1019200009F080E08F9300916200043680E010F0AF
:1019300009F081E09F91892B882311F40C947C0C91
:1019400000916200043618F011F00C94A90C0C946C
:10195000B80C81B5886181BD877F81BDE3E6F0E089
:10196000FA93EA930E943A0F229681B5886081BD6E
:1019700080E08093600081E090E00E94912E0091D1
:101980006000003011F00C94600C0C94060D009176
:10199000D200013011F00C94020D80E090E0A3E63B
:1019A000B0E08D939C93E0E6F0E0FA93EA930E9416
:1019B0002F1E2296A3E6B0E00E943F2DEF93FF93E7
:1019C000ECE8F1E00E94652EFF91EF91009160003C
:1019D000003081E009F080E08F93A3E6B0E00D9144
:1019E0001C91083250E0150780E010F009F081E00A
:1019F0009F91892B882311F40C94D30C81E090E003
:101A00000E94912E81E090E00E94912E0091D000E2
:101A1000003011F00C94100D85E090E00E94912EA2
:101A20000C9489020F921F922F923F924F925F92D5
:101A30007F928F929F92AF92BF920F931F932F939B
:101A40003F934F935F936F937F938F939F93AF9346
:101A5000BF93CF93DF93EF93FF938FB78F93F89458
:101A600089B78B7F89BF8EB5887F8EBD5A924A9287
:101A700080E092E0A42DB52D8D939C9382E00E948E
:101A80002C2D0E94A62C229682E00E94282D0091E7
:101A9000DB000A3011F00C944F0D0E94810E0E9461
:101AA00081250091DB000A3011F00C945C0D0E943E
:101AB000830E80E08093DB00ABEDB0E08C918F5F14
:101AC0008C93A8950027A1EDB0E08C9186FB0EF4D5
:101AD00001E040E0041711F00C94810D5A924A92F3
:101AE00080E092E0A42DB52D8D939C9382E00E941E
:101AF0002C2D0E94A62C229682E00E94282D0E9466
:101B00008125A7EDB0E04D915D916D917C91A3EDA4
:101B1000B0E00D911D912D913C910E94022F80E02B
:101B20000CF481E08F930027A1EDB0E08C9186FB4F
:101B30000EF401E040E0041781E009F080E09F919D
:101B40008923882311F40C94B00D80E49CE99DBD99
:101B50008CBD81E08EBD89B7846089BF0C94F90D7E
:101B600080E08093D00070916A00777F70936A0064
:101B70000027A1EDB0E08C9186FB0EF401E040E07F
:101B8000041711F00C94CD0DAAE6B0E08C9184FB03
:101B9000A8EBB0E0882780F98C930091C3004FE751
:101BA0000423A1E6B0E00C930E94830E80E08093B2
:101BB000C6000027A1EDB0E08C9183FB0EF401E09C
:101BC00041E0041781E009F080E08F930027A1ED48
:101BD000B0E08C9182FB0EF401E041E0041781E05B
:101BE00009F080E09F91892B882311F40C94F90D62
:101BF000DC988F918FBFFF91EF91DF91CF91BF91D3
:101C0000AF919F918F917F916F915F914F913F9194
:101C10002F911F910F91BF90AF909F908F907F90C9
:101C20005F904F903F902F901F900F901895F894D1
:101C3000FFCF89B78B7F89BF8EB5887F8EBD80E04F
:101C40008093D00070916A00777F70936A000027BC
:101C5000A1EDB0E08C9183FB0EF401E041E00417AC
:101C600081E009F080E08F930027A1EDB0E08C9136
:101C700082FB0EF401E041E0041781E009F080E00E
:101C80009F91892B882311F40C94470EDC980895BA
:101C9000DE9A6E98C498C598C7980E94830EE2E0B9
:101CA000F0E00E94EB2DDE98C49A0E947D2E84E61F
:101CB00090E00E94912EA8957091D1007F7B709347
:101CC000D100E0E6F0E0FA93EA930E944D222296DA
:101CD00000916000003011F40C947E0E7091D100E0
:101CE00070647093D10084E690E00E94912EDE9A99
:101CF0006E98C498C598C7980C94800E0E941415CD
:101D00000895AB980895AB9A089581E00E94A02EA3
:101D100070916A007F7E70936A000091C30041E079
:101D20000423A881B9810C93A881B9810C9100305A
:101D300011F40C94A00E70916A00706170936A00A7
:101D40007091D1007F777093D1000091C30042E081
:101D50000423A881B9810C93A881B9810C9100302A
:101D600011F40C94B80E7091D10070687093D1008A
:101D700070916A007E7F70936A000091C30044E016
:101D80000423A881B9810C93A881B9810C910030FA
:101D900011F40C94D00E70916A00716070936A0017
:101DA00070916A007D7F70936A000091C30048E0E3
:101DB0000423A881B9810C93A881B9810C910030CA
:101DC00011F40C94E80E70916A00726070936A00CE
:101DD00070916A007F7D70936A000091C30040E2B9
:101DE0000423A881B9810C93A881B9810C9100309A
:101DF00011F40C94000F70916A00706270936A0085
:101E00007091D1007F7E7093D1000091C40041E0B9
:101E10000423A881B9810C93A881B9810C91003069
:101E200011F40C94180F7091D10070617093D1006F
:101E30000091C40046E00423A881B9810C93A881D5
:101E4000B9810C9142E00E94A62F0C93A881B98120
:101E50008C918093D2000091D200033011F00C9449
:101E6000340F82E08093D20081E0481A8827580A14
:101E70002296089582E00E94A02E81E00E94A02E6A
:101E800081E00E94A02E80E0AA81BB818C9383E434
:101E9000ACE9B0E08C938FE4ADE9B0E08C938EE4D4
:101EA000AEE9B0E08C9386E4AFE9B0E08C9389E4CE
:101EB000A0EAB0E08C93AAE6B0E08C9185FBA88103
:101EC000B981882780F98C9370916A007062709351
:101ED0006A00A2E7B0E00D911D912D913C91A2E91D
:101EE000B0E00D931D932D933C935A924A92A2E930
:101EF000B0E00D911D912D913C91A42DB52D0D9328
:101F00001D932D933C9384E00E942C2D5A924A926B
:101F100080E090E0A42DB52D8D939C9382E00E94EB
:101F20002C2D5A924A9281E0A42DB52D8C9381E0FC
:101F30000E942C2D0E942316269687E00E94282DB1
:101F40008FE00E94A02EE4EAF0E006E0A881B981CB
:101F50000E947D2FA881B981E0E0F0E60E94B62FB3
:101F60000FB68FE0481A8827580A22960FBE81E0E4
:101F700009F080E08F9300918D00003181E009F03D
:101F800080E09F918923882311F40C94151081E03F
:101F9000AA81BB818C93A2E9B0E00D911D912D9196
:101FA0003C91A2E7B0E00D931D932D933C9370916B
:101FB0006A007F7D70936A005A924A92A2E9B0E06B
:101FC0000D911D912D913C91A42DB52D0D931D9337
:101FD0002D933C9384E00E942C2D5A924A9280E0EB
:101FE00090E0A42DB52D8D939C9382E00E942C2D22
:101FF0005A924A9280E0A42DB52D8C9381E00E94E4
:102000002C2D0E942316269687E00E94282DA2E9F7
:10201000B0E00D911D912D913C91A2E7B0E00D93A0
:102020001D932D933C930E946F10A881B9818C91D0
:1020300080FBAAE6B0E08C9185F98C93A6E7B0E02E
:102040000D911D912D913C91A2E7B0E00D931D9350
:102050002D933C93A2E7B0E00D911D912D913C9101
:10206000A2E9B0E00D931D932D933C935A924A92AE
:10207000A2E9B0E00D911D912D913C91A42DB52DBB
:102080000D931D932D933C9384E00E942C2D5A9226
:102090004A9280E090E0A42DB52D8D939C9382E030
:1020A0000E942C2D5A924A9280E0A42DB52D8C933B
:1020B00081E00E942C2D0E942316269687E00E9424
:1020C000282DAA81BB818C91AE81BF818D938827F9
:1020D0008C9384E0481A8827580A2696089582E04F
:1020E0000E94A02E81E00E94A02E81E00E94A02EDE
:1020F000789481E090E0AC81BD818D939C93EA81DE
:10210000FB81FA93EA93EE81FF81FA93EA930E94AE
:1021100085122496AA81BB810C91013011F00C9498
:102120009C1082E090E0AC81BD818D939C9381E016
:102130008093C3000C94B810023011F00C94AB10D3
:1021400083E090E0AC81BD818D939C9380E080938F
:10215000C3000C94B810033011F00C94B81084E054
:1021600090E0AC81BD818D939C9383E08093C3000C
:10217000EEE0F0E0A3ECB0E07BE70E948B2FEC8177
:10218000FD81FA93EA935A924A9280E0A42DB52DEC
:102190008C9381E00E942C2D0E94C212249681E033
:1021A0000E94282D0091D000003011F00C94D21024
:1021B00088EC90E00E94912E85E090E0AC81BD819A
:1021C0008D939C93EA81FB81FA93EA93EE81FF81E0
:1021D000FA93EA930E9485122496EEE0F0E0A3ECD5
:1021E000B0E00E949C2FAA81BB810C91033011F0BA
:1021F0000C94FC100C949911AA81BB810C910130B4
:1022000011F00C940A11A3ECB0E08C9188608C93CF
:102210000C941311023011F00C941311A3ECB0E0E4
:102220008C91877F8C93EEE0F0E0A3ECB0E07BE74D
:102230000E948B2F88EC90E00E94912E86E090E027
:10224000AC81BD818D939C93EA81FB81FA93EA93E3
:10225000EE81FF81FA93EA930E9485122496AA8167
:10226000BB810C91033011F00C9438110C9499112E
:10227000EEE0F0E0A3ECB0E00E949C2FAA81BB81CD
:102280000C91013011F00C944C11A3ECB0E08C9146
:1022900084608C930C945511023011F00C945511FC
:1022A000A3ECB0E08C918B7F8C93EEE0F0E0A3EC9C
:1022B000B0E07BE70E948B2F88EC90E00E94912E8B
:1022C00087E090E0AC81BD818D939C93EA81FB8196
:1022D000FA93EA93EE81FF81FA93EA930E948512C2
:1022E0002496EEE0F0E0A3ECB0E00E949C2FAA81DF
:1022F000BB810C91013011F00C948511A3ECB0E07E
:102300008C9180628C930C948E11023011F00C949D
:102310008E11A3ECB0E08C918F7D8C93EEE0F0E019
:10232000A3ECB0E07BE70E948B2F88EC90E00E944A
:10233000912E88E090E0AC81BD818D939C93EC81DF
:10234000FD81FA93EA930E94631222960091C300E2
:1023500043E00423A881B9810C93A881B9810C9131
:10236000003011F00C94BC1183E090E0AC81BD8191
:102370008D939C930C94D211013011F00C94C811E0
:1023800082E090E0AC81BD818D939C930C94D2113E
:10239000033011F00C94D21184E090E0AC81BD8147
:1023A0008D939C93EC81FD81FA93EA930E946312D2
:1023B00022960091C30048E00423A881B9810C93C0
:1023C000A881B9810C91003011F00C94EF118AE0D2
:1023D00090E0AC81BD818D939C930C94F9110830F1
:1023E00011F00C94F91189E090E0AC81BD818D93DE
:1023F0009C93EC81FD81FA93EA930E9463122296EA
:102400000091C30044E00423A881B9810C93A88102
:10241000B9810C91003011F00C9416128BE090E011
:10242000AC81BD818D939C930C942012043011F0EB
:102430000C9420128CE090E0AC81BD818D939C9334
:10244000EC81FD81FA93EA930E9463122296009137
:10245000C30040E20423A881B9810C93A881B9810B
:102460000C91003011F00C943D128DE090E0AC81A5
:10247000BD818D939C930C944712003211F00C9403
:1024800047128EE090E0AC81BD818D939C93EC81EE
:10249000FD81FA93EA930E94631222968FE090E006
:1024A000AC81BD818D939C93EC81FD81FA93EA937D
:1024B0000E94631222960E94850E84E0481A8827A3
:1024C000580A26960895E881F981FA93EA935A9278
:1024D0004A9280E0A42DB52D8C9381E00E942C2D92
:1024E0000E94C212249681E00E94282D82E390E08F
:1024F0000E94912E0091D000003011F00C947A12BD
:1025000082E390E00E94912E089581E00E94A02E27
:10251000EA81FB81FA93EA935A924A9280E0A42DD1
:10252000B52D8C9381E00E942C2D0E94C21224961E
:1025300081E00E94282D84E690E00E94912EE8819F
:10254000F981FA93EA930E94D71D2296A881B98156
:102550000C91003018F011F00C94B0120C949F12F2
:102560000E94190E84E190E00E94912EA881B98109
:102570008C91AC81BD818C9381E0481A8827580AE0
:102580002296089582E00E94A02E81E00E94A02E53
:102590008EB5887F8EBD70916A00777F70936A00D8
:1025A000A2E7B0E00D911D912D913C91A2E9B0E020
:1025B0000D931D932D933C935A924A92A2E9B0E059
:1025C0000D911D912D913C91A42DB52D0D931D9331
:1025D0002D933C9384E00E942C2D5A924A92AA8516
:1025E000BB858D919C91A42DB52D8D939C9382E0FC
:1025F0000E942C2D5A924A9280E0A42DB52D8C93E6
:1026000081E00E942C2D0E942316269687E00E94CE
:10261000282D40E050E060E070E0AEE8B0E00D91C1
:102620001D912D913C910E94022F11F00C941A13D0
:102630000C940E150E94EF285A924A928091BB008A
:10264000A42DB52D8C9381E00E942C2D5A924A9294
:102650008091C000A42DB52D8C9381E00E942C2D7B
:102660005A924A928091C100A42DB52D8C9381E09D
:102670000E942C2D0E943B29269683E00E94282D43
:102680005A924A92ACEBB0E08D919C91A42DB52D5D
:102690008D939C9382E00E942C2D0E94422A2296C8
:1026A00082E00E94282D0027A1EDB0E08C9184FBF0
:1026B0000EF401E041E0041711F00C9479135A92E2
:1026C0004A928091BE00A42DB52D8C9381E00E948A
:1026D0002C2D5A924A928091BF00A42DB52D8C9337
:1026E00081E00E942C2D0E94032A249682E00E9401
:1026F000282DA2E9B0E00D911D912D913C91A3ED03
:10270000B0E00D931D932D933C93A2E9B0E00D91A1
:102710001D912D913C91AEE8B0E04D915D916D9190
:102720007C910E94F82EA7EDB0E00D931D932D93A0
:102730003D9380E0A881B9818C930E94812581E03E
:1027400090E0AA81BB818D939C93AA81BB810D915E
:102750001C910F3F51E0150718F011F00C94DF1396
:10276000AA81BB81AD90BC90ABEDB0E0AA0DBB1DC2
:102770000C910F3F81E009F080E08F93AA81BB812B
:10278000AD90BC90ACEDB0E0AA0DBB1D0C910F3E1E
:1027900080E010F009F081E09F918923882311F4F3
:1027A0000C94D81381E0A881B9818C930C94DF1329
:1027B000AA81BB810E943F2D11F00C94A513A88122
:1027C000B9810C91013011F00C949D13AA81BB8149
:1027D000AD90BC90ADEDB0E0AA0DBB1D8C91AA816F
:1027E000BB818D9388278C93AA81BB810D911C910D
:1027F00040E150E00E94712DAA81BB814D935C9312
:1028000080E18093C500AA81BB810D911C910130AC
:1028100050E0150711F00C94121484E08093C50069
:102820000C949F14023050E0150711F00C941D1405
:1028300085E08093C5000C949F14033050E0150789
:1028400011F00C94281486E08093C5000C949F141A
:10285000043050E0150711F00C94331487E0809396
:10286000C5000C949F14053050E0150711F00C942E
:102870003E1488E08093C5000C949F14063050E00D
:10288000150711F00C9449148AE08093C5000C944C
:102890009F14073050E0150711F00C9454148CE08D
:1028A0008093C5000C949F14083050E0150711F078
:1028B0000C945F148EE08093C5000C949F14093033
:1028C00050E0150711F00C946A1480E18093C50064
:1028D0000C949F140A3050E0150711F00C947514F5
:1028E00084E18093C5000C949F140B3050E01507D1
:1028F00011F00C94801488E18093C5000C949F140F
:102900000C3050E0150711F00C948B148CE180937F
:10291000C5000C949F140D3050E0150711F00C9475
:10292000961480E28093C5000C949F140E3050E002
:10293000150711F00C949F1488E28093C500AEE84F
:10294000B0E00D911D912D913C9140E052E060E08E
:1029500070E00E94F12DA5E6B0E00D931D932D933C
:102960003D93A5E6B0E00D911D912D913C91A5EC14
:10297000B0E04C915527662777270E94F62DA5E6F3
:10298000B0E04D935D936D937D93A5E6B0E00D911E
:102990001D912D913C9148EE53E060E070E00E9463
:1029A000F62DA5E6B0E04D935D936D937D93AC81DC
:1029B000BD810C91003011F00C940E1581E08093D4
:1029C000D00088EC9FEA9DBD8CBD89B7846089BF2B
:1029D00081E08EBD0027A1EDB0E08C9183FB0EF469
:1029E00001E041E0041781E009F080E08F930027C7
:1029F000A1EDB0E08C9182FB0EF401E041E0041700
:102A000081E009F080E09F91892B882311F40C94D8
:102A10000A15DC9A85E090E00E94912E83E0481A26
:102A20008827580A24960895A895A2E7B0E00D914A
:102A30001D912D913C91A6E7B0E00D931D932D9330
:102A40003C93A2E7B0E00D911D912D913C91A2E93C
:102A5000B0E00D931D932D933C935A924A92A2E9B4
:102A6000B0E00D911D912D913C91A42DB52D0D93AC
:102A70001D932D933C9384E00E942C2D5A924A92F0
:102A800080E090E0A42DB52D8D939C9382E00E9470
:102A90002C2D5A924A9280E0A42DB52D8C9381E082
:102AA0000E942C2D0E942316269687E00E94282D36
:102AB000A895A2EBB0E00D911C91013050E01507F4
:102AC00010F00C948A155A924A9281E0A42DB52DEB
:102AD0008C9381E00E942C2D0E949C2A229681E0FA
:102AE0000E94282D8CE291E00E94912E5A924A92E7
:102AF00080E0A42DB52D8C9381E00E942C2D0E94A6
:102B00009C2A229681E00E94282D7091D100706449
:102B10007093D100A895A2E7B0E00D911D912D9181
:102B20003C91A2E9B0E00D931D932D933C93A6EB4D
:102B3000B0E00D911C91003050E0150781E009F0E4
:102B400080E08F93A2EBB0E04D915C91A6EBB0E0FA
:102B50000D911C910417150780E010F009F081E039
:102B60009F91892B882311F40C94BC1581E090E08F
:102B7000A6EBB0E08D939C930E94830E089584E0B1
:102B80000E94A02EA3EDB0E00D911D912D913C91DE
:102B9000A881B9810D931D932D933C93A2E7B0E0DA
:102BA0000D911D912D913C91A2E9B0E00D931D93E3
:102BB0002D933C935A924A92A2E9B0E00D911D9157
:102BC0002D913C91A42DB52D0D931D932D933C93E8
:102BD00084E00E942C2D5A924A928FE19EE4A42D0B
:102BE000B52D8D939C9382E00E942C2D5A924A928F
:102BF00080E0A42DB52D8C9381E00E942C2D0E94A5
:102C00002316269687E00E94282DA2E7B0E00D91BA
:102C10001D912D913C91A2E9B0E00D931D932D9350
:102C20003C93A881B9810D911D912D913C91A3ED0B
:102C3000B0E00D931D932D933C9384E0481A8827B0
:102C4000580A2296089581E00E94A02E81E00E94F9
:102C5000A02E81E00E94A02E80E090E0A4EBB0E0E6
:102C60008D939C9370916A007F7B70936A0000E063
:102C700010E020E030E0AEE8B0E00D931D932D931E
:102C80003C930027AAE6B0E08C9185FB0EF401E0AE
:102C900041E0041781E009F080E08F93A885B985B1
:102CA0000D911C91003050E0150781E009F480E09F
:102CB0009F9189238F93AE81BF810C91003081E079
:102CC00009F080E09F918923882311F40C94C316A6
:102CD000A6E9B0E0E885F9850E94152FE6E9F0E065
:102CE000A8E6B7E00E94712FE8E6F7E0A6E9B0E0B9
:102CF0001127222704E033270E94BA2E81E4AC81F9
:102D0000BD818C93AC81BD818C9180939C0081E0CE
:102D1000E6E9F0E001E00A93ABE6B0E00E94762F2E
:102D2000ABE6B0E08C91ADE9B0E08C9382E0E6E9EF
:102D3000F0E001E00A93ABE6B0E00E94762FABE64C
:102D4000B0E08C91AEE9B0E08C9383E0E6E9F0E08E
:102D500001E00A93ABE6B0E00E94762FABE6B0E06C
:102D60008C91AFE9B0E08C9384E0E6E9F0E001E01B
:102D70000A93ABE6B0E00E94762FABE6B0E08C9110
:102D8000A0EAB0E08C9389B78B7F89BF8EB5887F2E
:102D90008EBD81B5886181BD877F81BDACECB0E01F
:102DA0000D911D912D913C91A8ECB0E00D931D93D8
:102DB0002D933C93A6E7B0E04D915D916D917C9190
:102DC000A2E7B0E00D911D912D913C910E94022F40
:102DD00011F00C94F51602E010E020E030E0A8ECD1
:102DE000B0E00D931D932D933C9380E0A881B981B1
:102DF0008C93EA81FB81FA93EA935A924A92AE85C8
:102E0000BF850D911D912D913C91A42DB52D0D9354
:102E10001D932D933C9384E00E942C2D0E947827D3
:102E2000249684E00E94282DAA81BB810C910E3F3C
:102E300011F40C9427177091D10070647093D10035
:102E400070916A00706470936A000C943A175A92F9
:102E50004A92AA85BB858D919C91A42DB52D8D9309
:102E60009C9382E00E942C2D0E943B18229682E0C7
:102E70000E94282DA881B9818C918F5F8C934091FD
:102E80006F00A881B9810C91041781E009F080E0FE
:102E90008F930027AAE6B0E08C9186FB0EF401E048
:102EA00041E0041781E009F480E09F9189238823A1
:102EB00011F40C94F01700917E000B3011F00C947B
:102EC0009D17E8ECF0E0FA93EA935A924A92A8EC44
:102ED000B0E00D911D912D913C91A42DB52D0D9338
:102EE0001D932D933C9384E00E942C2D0E947B1C0B
:102EF000249684E00E94282DEA85FB85FA93EA93C4
:102F00005A924A92A8ECB0E00D911D912D913C91FE
:102F1000A42DB52D0D931D932D933C9384E00E9419
:102F20002C2D0E94111C249684E00E94282D80E004
:102F3000A881B9818C930C94EE17A6E7B0E04D916F
:102F40005D916D917C91A2E7B0E00D911D912D9165
:102F50003C910E94022F11F00C94B417AA85BB85F6
:102F60000E94302D0C94EE17E8ECF0E0FA93EA930F
:102F70005A924A92A8ECB0E00D911D912D913C918E
:102F8000A42DB52D0D931D932D933C9384E00E94A9
:102F90002C2D0E947B1C249684E00E94282DEA851B
:102FA000FB85FA93EA935A924A92A8ECB0E00D910D
:102FB0001D912D913C91A42DB52D0D931D932D9315
:102FC0003C9384E00E942C2D0E94111C249684E0E6
:102FD0000E94282D80E0A881B9818C930C94F4176D
:102FE000AA85BB850E94302D0027AAE6B0E08C910F
:102FF00086FB0EF401E041E0041711F00C94F91681
:10300000C49AA885B9850D911C91003050E0150730
:1030100011F00C941318A4EBB0E08D919C91A2EBED
:10302000B0E08D939C930091D000013081E009F0D5
:1030300080E08F930027A1EDB0E08C9186FB0EF429
:1030400001E040E0041781E009F080E09F918923CE
:10305000882311F40C94351880E593EC9DBD8CBD4C
:1030600081E08EBD89B7846089BF83E0481A8827D4
:10307000580A2696089584E00E94A02E84E00E94BB
:10308000A02E81E00E94A02E81E00E94A02E81E06F
:103090000E94A02E81E00E94A02E80E0AE81BF8120
:1030A0008C93AE81BF810C910F3018F011F00C940D
:1030B0001E1A81E0AC81BD818C93AC81BD810C91E5
:1030C0000C3018F011F00C947D188FEF0E94842EB4
:1030D0000E94862E0E94852EAC81BD81AD90BB24BE
:1030E000A0E8B0E0AA0DBB1D8C93AC81BD818C9192
:1030F0008F5F8C9311F00C945D188DE0AC81BD81D5
:103100008C93AC81BD810C91043118F011F00C94BA
:103110009B188FEF0E94842E0E94862E0E94852E7F
:10312000A881B9818C93AC81BD818C918F5F8C9388
:1031300011F00C948118EA85FB85FA93EA93EA85ED
:10314000FB85FA93EA930E94A61A24960027AAE622
:10315000B0E08C9186FB0EF401E041E0041711F021
:103160000C94B4180C94161A80E0AA81BB818C933D
:1031700000918C00003281E009F080E08F93009193
:103180008C00003181E009F080E09F91892B882339
:1031900011F40C94CF1881E0AA81BB818C9300912B
:1031A0008100003081E009F480E08F93009181007C
:1031B000053E81E009F480E09F9189238F93AA81E5
:1031C000BB810C91013081E009F080E09F9189235F
:1031D000882311F40C940B1A00918C00003211F02A
:1031E0000C94F618A4EBB0E00E943F2D0027AAE64D
:1031F000B0E08C9185FB0EF401E040E0041711F083
:103200000C942B1981E0AC81BD818C93AC85BD857C
:103210004D915C91A4EBB0E00D911C910417150742
:1032200081E009F080E08F93A4EBB0E00D911C9158
:10323000003050E0150780E010F009F081E09F9128
:103240008923882311F40C94291980E0AC81BD8175
:103250008C930C945F1980E0AC81BD818C9381E0EC
:10326000A881B9818C93A881B9810C91053018F09F
:1032700011F00C945F19A881B981AD90BB24ABE922
:10328000B0E0AA0DBB1D4C91A881B981AD90BB24C3
:10329000A0E8B0E0AA0DBB1D0C91041711F40C942A
:1032A000571981E0AC81BD818C930C945F19A88182
:1032B000B9818C918F5F8C9311F00C943319AC8190
:1032C000BD810C91003081E009F080E08F93AC85E6
:1032D000BD850D911C910F315EE4150781E009F069
:1032E00080E09F91892B882311F40C940B1A0E9483
:1032F000381AA885B9850D911D912D913C9140E01A
:1033000052E060E070E00E94F62DAEE8B0E04D9330
:103310005D936D937D93E2E9F0E0FA93EA935A921C
:103320004A92AE85BF850D911D912D913C91A42DA2
:10333000B52D0D931D932D933C9384E00E942C2D6D
:103340000E94111C249684E00E94282D80918C00FC
:1033500080938D00AC85BD850D911C910F315EE48D
:10336000150711F00C94DC19A8E6B7E0E4EBF0E0E7
:103370000E94152F0E94D02DE8E0F0E60E94D82D83
:10338000A4EAB0E00E94D22DE8E0F0E60E94D82D39
:1033900000918C00003111F00C94D219EAE0F0E6B3
:1033A0000E94D82DA8E6B7E0E885F9850E94182F7D
:1033B0000E94D02D0E94E42DAC81BD810C91003083
:1033C00011F00C940B1A70916A00706470936A008B
:1033D00000918D00003181E009F080E08F93AC8591
:1033E000BD850D911C910F315EE4150781E009F454
:1033F00080E09F918923882311F40C940B1AAA85ED
:10340000BB850D911D912D913C91ACECB0E00D93DD
:103410001D932D933C9300918100003011F00C948A
:10342000161A70916A00706470936A00AE81BF8151
:103430008C918F5F8C9311F00C9451188FEF0E9438
:10344000842E0E94862E0E94852EA0E6B0E08C93EA
:103450008FEF0E94842E0E94862E0E94852EA0E669
:10346000B0E08C938CE0481A8827580A2C9608956F
:1034700081E00E94A02EA4EAB0E088278C9381E02E
:10348000A881B9818C93A881B9810C91083018F07A
:1034900011F00C94721AA881B981AD90BB24A0E8F8
:1034A000B0E0AA0DBB1D0C91003211F40C946A1A05
:1034B000A881B981AD90BB24A0E8B0E0AA0DBB1DE6
:1034C0008C91A4EAB0E08F930E94BD2D8F918D93D3
:1034D00088278C93A881B9818C918F5F8C9311F090
:1034E0000C94431AA4EAB0E00E94BD2DEEE0F0E691
:1034F0000E94B72D89E0A881B9818C93A881B981F8
:103500000C910B3018F011F00C94A01AA881B9811D
:10351000AD90BB24A0E8B0E0AA0DBB1D8C91A4EA3D
:10352000B0E08F930E94BD2D8F918D9388278C934F
:10353000A881B9818C918F5F8C9311F00C947E1AC5
:1035400081E0481A8827580A2296089581E00E944F
:10355000A02E81E00E94A02E84E00E94A02E8FEF7A
:103560000E94842E0E94862E0E94852EAC81BD81F1
:103570008C938FEF0E94842E0E94862E0E94852EAF
:10358000AA81BB818C93AA81BB810C911127222730
:10359000332740E051E060E070E00E94F12DA88503
:1035A000B9850D931D932D933D93A885B9850D91F4
:1035B0001D912D913C91AC81BD814C915527662781
:1035C00077270E94F82EA885B9850D931D932D931A
:1035D0003D93A885B9850D911D912D913C9140E0B9
:1035E00050E061E070E00E94F12DA881B9810D9357
:1035F0001D932D933D938FEF0E94842E0E94862E63
:103600000E94852EAC81BD818C938FEF0E94842E09
:103610000E94862E0E94852EAC81BD818C938FEFF7
:103620000E94842E0E94862E0E94852EAC81BD8130
:103630008C938FEF0E94842E0E94862E0E94852EEE
:10364000AC81BD818C938FEF0E94842E0E94862EC8
:103650000E94852EAC81BD818C938FEF0E94842EB9
:103660000E94862E0E94852EAA81BB818C93AA81FE
:10367000BB810C9111272227332740E051E060E005
:1036800070E00E94F12DA885B9850D931D932D93AF
:103690003D93A885B9850D911D912D913C91AC81EB
:1036A000BD814C915527662777270E94F82EA88563
:1036B000B9850D931D932D933D93A885B9850D91E3
:1036C0001D912D913C91A881B9814D915D916D9194
:1036D0007C910E94F82EA885B9850D931D932D939A
:1036E0003D938FEF0E94842E0E94862E0E94852E8D
:1036F000AC81BD818C938FEF0E94842E0E94862E18
:103700000E94852EAA81BB818C93AA81BB810C91DA
:1037100011272227332740E051E060E070E00E944B
:10372000F12DA881B9810D931D932D933D93A8810F
:10373000B9810D911D912D913C91AC81BD814C9130
:103740005527662777270E94F82EA881B9810D9307
:103750001D932D933D938FEF0E94842E0E94862E01
:103760000E94852EAC81BD818C938FEF0E94842EA8
:103770000E94862E0E94852EAA81BB818C93AA81ED
:10378000BB810C9111272227332740E051E060E0F4
:1037900070E00E94F12DAE81BF810D931D932D939A
:1037A0003D93AE81BF810D911D912D913C91AC81D6
:1037B000BD814C915527662777270E94F82EAE8150
:1037C000BF810D931D932D933D93AE81BF810D91CC
:1037D0001D912D913C9140E050E061E070E00E942D
:1037E000F12DAE81BF810D931D932D933D93AE813D
:1037F000BF810D911D912D913C91A881B9814D9171
:103800005D916D917C910E94F82EAE81BF810D93E8
:103810001D932D933D9386E0481A8827580A2696D3
:10382000089584E00E94A02E84E00E94A02EAC8126
:10383000BD810D911D912D913C9142E050E060E0E1
:1038400070E00E94FD2EA881B9810D931D932D93E8
:103850003D93AFE6B0E00C91112722273327A881D2
:10386000B9814D915D916D917C910E94F12DAA815C
:10387000BB810D931D932D933D93AA81BB810D9127
:103880001D912D913C91A6E7B0E04D915D916D9118
:103890007C910E94F82EAA81BB810D931D932D93DC
:1038A0003D9300917E000B3011F40C94691CAA81A9
:1038B000BB810D911D912D913C9140E250E060E063
:1038C00070E00E94F82EAA81BB810D931D932D9369
:1038D0003D93AA81BB810D911D912D913C91AE81AB
:1038E000BF810D931D932D933C9388E0481A882740
:1038F000580A2496089584E00E94A02E82E00E9437
:10390000A02E00917E000B3011F00C94BF1CAC81F6
:10391000BD810D911D912D913C9140E850E060E0FA
:1039200070E00E94F62DA3EDB0E04D935D936D9392
:103930007D93AC81BD810D911C9140E850E00E94C7
:10394000912DA881B9810D931C93A881B9810D9106
:103950001C9144E050E00E94AB2DA881B9810D93E9
:103960001C93A881B9810D911C9144E050E0040F93
:10397000151FA881B9810D931C930C94F51CAC8183
:10398000BD810D911D912D913C9140E051E060E091
:1039900070E00E94F62DA3EDB0E04D935D936D9322
:1039A0007D93AC81BD810D911C9140E051E00E945E
:1039B000912DA881B9810D931C93A881B9810D9196
:1039C0001C9142E050E00E94AB2DA881B9810D937B
:1039D0001C93A881B9810D911C9142E050E0040F25
:1039E000151FA881B9810D931C93A3EDB0E00D9133
:1039F0001D912D913C91AAE7B0E04D915D916D91A3
:103A00007C910E94F82EA3EDB0E00D931D932D93B1
:103A10003D93A3EDB0E00D911D912D913C91ADE64C
:103A2000B0E04D915C91662777270E94F82EA3EDB8
:103A3000B0E00D931D932D933D930E948125A881A5
:103A4000B981AD90BC90ABEDB0E0AA0DBB1D8C91DF
:103A5000AA81BB818D9388278D938D938C93A881A8
:103A6000B9810E94452DAA81BB810D911D912D9197
:103A70003C9140E051E060E070E00E94F12DAA81AD
:103A8000BB810D931D932D933D93AA81BB810D9115
:103A90001D912D913C91A881B981AD90BC90ABED69
:103AA000B0E0AA0DBB1D4C915527662777270E94D1
:103AB000F82EAA81BB810D931D932D933D93009108
:103AC0007E000B3011F00C94C51DA881B9810E94B5
:103AD000452DAA81BB810D911D912D913C9140E016
:103AE00051E060E070E00E94F12DAA81BB810D934E
:103AF0001D932D933D93AA81BB810D911D912D9115
:103B00003C91A881B981AD90BC90ABEDB0E0AA0D1D
:103B1000BB1D4C915527662777270E94F82EAA8156
:103B2000BB810D931D932D933D93A881B9810E9474
:103B3000452DAA81BB810D911D912D913C9140E0B5
:103B400051E060E070E00E94F12DAA81BB810D93ED
:103B50001D932D933D93AA81BB810D911D912D91B4
:103B60003C91A881B981AD90BC90ABEDB0E0AA0DBD
:103B7000BB1D4C915527662777270E94F82EAA81F6
:103B8000BB810D931D932D933D93AA81BB810D9114
:103B90001D912D913C91AE81BF810D931D932D936D
:103BA0003C9386E0481A8827580A2496089580E0B6
:103BB000A881B9818C930027BB27A0E38C9183FB5C
:103BC0000EF401E040E0041711F00C94EB1D82E0CC
:103BD000A881B9818C930027BB27A0E38C9184FB3B
:103BE0000EF401E040E0041711F00C94FB1D81E09D
:103BF000A881B9818C930027BB27A3E38C9181FB1B
:103C00000EF401E040E0041711F00C940B1E83E069
:103C1000A881B9818C930027BB27A3E38C9181FBFA
:103C20000EF401E040E0041781E009F080E08F939A
:103C30000027BB27A0E38C9183FB0EF401E040E05A
:103C4000041781E009F080E09F918923882311F413
:103C50000C942E1E84E0A881B9818C93089581E094
:103C60000E94A02E81E00E94A02E82E00E94A02E41
:103C70000027A1EDB0E08C9183FB0EF401E041E060
:103C8000041711F00C945A1E80E0AC81BD818C9316
:103C90000027BB27A9E38C9185FB0EF401E040E0EF
:103CA000041711F00C94581E81E0AC81BD818C93F7
:103CB0000C945A1F5398549880E081BB909A919A23
:103CC000EF93FF93E0EFF1E00E94652EFF91EF91FB
:103CD00080E0AC81BD818C930027BB27A0E38C9151
:103CE00080FB0EF401E040E0041711F00C947C1E00
:103CF00081E0AC81BD818C930027BB27A0E38C9130
:103D000081FB0EF401E040E0041711F00C948D1ECD
:103D1000AC81BD818C918E5F8C930027BB27A9E37A
:103D20008C9185FB0EF401E040E0041711F00C9437
:103D30009E1EAC81BD818C918C5F8C930027BB272C
:103D4000A9E38C9184FB0EF401E040E0041711F02C
:103D50000C94AF1EAC81BD818C91885F8C93AC813B
:103D6000BD810C91003018F011F00C94B91E0C9428
:103D7000121F85E090E00E94912E80E0AA81BB8115
:103D80008C930027BB27A0E38C9180FB0EF401E00D
:103D900040E0041711F00C94D11E81E0AA81BB8190
:103DA0008C930027BB27A0E38C9181FB0EF401E0EC
:103DB00040E0041711F00C94E21EAA81BB818C91A3
:103DC0008E5F8C930027BB27A9E38C9185FB0EF4B3
:103DD00001E040E0041711F00C94F31EAA81BB81AE
:103DE0008C918C5F8C930027BB27A9E38C9184FB7B
:103DF0000EF401E040E0041711F00C94041FAA81B6
:103E0000BB818C91885F8C93AA81BB814C91AC81E2
:103E1000BD810C91041711F40C94121F80E0AC8149
:103E2000BD818C93AC81BD810C91033011F00C9459
:103E30001F1F82E0AC81BD818C930C94551FAC8117
:103E4000BD810C91043081E008F480E08F93AC8157
:103E5000BD810C91073081E010F009F080E09F9166
:103E60008923882311F40C943B1F83E0AC81BD812E
:103E70008C930C94551FAC81BD810C91083081E06E
:103E800008F480E08F93AC81BD810C910F3081E00C
:103E900010F009F080E09F918923882311F40C949D
:103EA000551F84E0AC81BD818C9381E081BB9198EA
:103EB000539A549AAC81BD818C91AE81BF818C9311
:103EC00084E0481A8827580A2696089581E00E94BF
:103ED000A02E81E00E94A02EAC81BD818C91A88192
:103EE000B9818C930E94810E88EC90E00E94912E03
:103EF0005A924A9281E0A42DB52D8C9381E00E94C4
:103F00002C2D0E949C2A229681E00E94282DA895A3
:103F1000E9E6F0E0FA93EA930E94D71D22968AE040
:103F200090E00E94912E00916900003011F00C94F5
:103F3000871F86E990E00E94912E5A924A9280E073
:103F4000A42DB52D8C9381E00E942C2D0E949C2ADB
:103F5000229681E00E94282D84E690E00E94912E16
:103F60005A924A9280E0A42DB52D8C9381E00E9454
:103F70002C2D0E949C2A229681E00E94282DA89533
:103F8000E9E6F0E0FA93EA930E94D71D22960E9498
:103F9000830E5A924A9281E0A42DB52D8C9381E034
:103FA0000E942C2D0E949C2A229681E00E94282D9E
:103FB00084E690E00E94912E5A924A9280E0A42DCD
:103FC000B52D8C9381E00E942C2D0E949C2A229674
:103FD00081E00E94282D8AE090E00E94912E5A9262
:103FE0004A9280E0A42DB52D8C9381E00E942C2D67
:103FF0000E949C2A229681E00E94282D0E94810E18
:1040000086E990E00E94912E00916900003018F03E
:1040100011F00C940D200C94BF1F88E790E00E94D3
:10402000912E5A924A9281E0A42DB52D8C9381E075
:104030000E942C2D0E942E21229681E00E94282D84
:10404000A881B9810C91023011F00C946720009185
:104050006900013011F00C94322081E08093C3009C
:104060000C946020023011F00C944A2080E0809380
:10407000C3005A924A9281E0A42DB52D8C9381E021
:104080000E942C2D0E942E21229681E00E94282D34
:104090000C946020033011F00C94602083E0809336
:1040A000C3005A924A9282E0A42DB52D8C9381E0F0
:1040B0000E942C2D0E942E21229681E00E94282D04
:1040C000EEE0F0E0A3ECB0E07BE70E948B2FA8814C
:1040D000B9810C91033011F00C949A200091690081
:1040E000013011F00C947B20A4ECB0E08C91816045
:1040F0008C930C949320023011F00C949320A4EC38
:10410000B0E08C918E7F8C935A924A9281E0A42DDC
:10411000B52D8C9381E00E942C2D0E942E21229699
:1041200081E00E94282DEFE0F0E0A4ECB0E07BE716
:104130000E948B2FA881B9810C91013011F00C9451
:10414000EC2000916900013011F00C94B320A4EC34
:10415000B0E08C9182608C93A4ECB0E08C918B7F6A
:104160008C930C94E520023011F00C94CD20A4EC3B
:10417000B0E08C91897F8C935A924A9281E0A42D71
:10418000B52D8C9381E00E942C2D0E942E21229629
:1041900081E00E94282D0C94E520033011F00C944E
:1041A000E520A4ECB0E08C9186608C935A924A9200
:1041B00082E0A42DB52D8C9381E00E942C2D0E94CD
:1041C0002E21229681E00E94282DEFE0F0E0A4EC61
:1041D000B0E07BE70E948B2F0E94850EA895E9E650
:1041E000F0E0FA93EA930E94D71D229685E090E0D2
:1041F0000E94912E00916900003011F00C94EE2085
:1042000086E990E00E94912E5A924A9280E0A42D75
:10421000B52D8C9381E00E942C2D0E949C2A229621
:1042200081E00E94282D86E990E00E94912E5A920A
:104230004A9280E0A42DB52D8C9381E00E942C2D14
:104240000E949C2A229681E00E94282D0E94830EC3
:1042500082E0481A8827580A2496089581E00E942F
:10426000A02E81E0A881B9818C93AA81BB814C9159
:10427000A881B9810C91041718F011F00C945B21FE
:104280005A924A9282E0A42DB52D8C9381E00E942F
:104290002C2D0E949C2A229681E00E94282D8DE7D9
:1042A00090E00E94912EA881B9818C918F5F8C93B0
:1042B00011F00C94352181E0481A8827580A22967B
:1042C000089581E00E94A02E81E0A881B9818C939D
:1042D000A881B9810C91063018F011F00C9484215A
:1042E0000E94810E8FE090E00E94912E0E94830E2A
:1042F00084E690E00E94912EA881B9818C918F5F15
:104300008C9311F00C94682181E0481A8827580A90
:104310002296089580E08093C00080E08093C100E1
:104320000E947D2EC39A88EC90E00E94912E81B568
:10433000886081BD0E94EF285A924A9281E0A42DA4
:10434000B52D8C9381E00E942C2D5A924A92809137
:10435000C000A42DB52D8C9381E00E942C2D5A9283
:104360004A928091C100A42DB52D8C9381E00E94CA
:104370002C2D0E943B29269683E00E94282D81B592
:10438000886181BD877F81BD84E690E00E94912E87
:10439000FF27E0E1FA93EA935A924A928BE0A42D28
:1043A000B52D8C9381E00E942C2D0E94322C2496F6
:1043B00081E00E94282D013051E0150711F00C9486
:1043C000FA215A924A92ACEBB0E08D919C91A42DC7
:1043D000B52D8D939C9382E00E942C2D0E94422A41
:1043E000229682E00E94282DE0E1F0E60E94D82D7E
:1043F0000E94E42D5A924A9282E3A42DB52D8C930B
:1044000081E00E942C2D5A924A928091C000A42DE6
:10441000B52D8C9381E00E942C2D5A924A92809166
:10442000C100A42DB52D8C9381E00E942C2D0E94FB
:104430003B29269683E00E94282DC29AD89A82E3CF
:1044400090E00E94912E089581E00E94A02E81E0CC
:104450000E94A02E8FEFAA81BB818C9380E0A8815F
:10446000B9818C93A881B9810C91073018F011F0B3
:104470000C94472291E0AA81BB810E94732EA881EF
:10448000B9818C918F5F8C9311F00C94322282E071
:10449000481A8827580A2496089581E00E94A02E81
:1044A00081E00E94A02E81E00E94A02E82E00E9466
:1044B000A02E82E00E94A02E8FEFAA85BB858C9350
:1044C00081E0A885B9858C93A885B9850C910034C5
:1044D00018F011F00C9476220E942422A885B98548
:1044E0008C918F5F8C9311F00C946422C49881E0BE
:1044F000A885B9858C93A885B9850C91003418F0EE
:1045000011F00C948D220E942422A885B9858C91EB
:104510008F5F8C9311F00C947B228AE090E00E94D4
:10452000912EA895EE81FF81FA93EA935A924A92CE
:1045300080E4A42DB52D8C9381E00E942C2D5A92FD
:104540004A9200E010E020E030E0A42DB52D0D935C
:104550001D932D933C9384E00E942C2D0E945E2895
:10456000269685E00E94282DAE81BF810C910130F6
:1045700011F40C94C422C49AE4E1F0E60E94D82D10
:104580000E94E42D0C947B2581E0AA85BB858C9349
:10459000A89580E090E0A881B9818D939C93EE81ED
:1045A000FF81FA93EA935A924A9281E4A42DB52DA1
:1045B0008C9381E00E942C2D5A924A9200E010E0E8
:1045C00020E030E0A42DB52D0D931D932D933C9349
:1045D00084E00E942C2D0E945E28269685E00E9491
:1045E000282DA881B9810E943F2DAE81BF810C91F9
:1045F000003081E009F080E08F93A881B9810D91AE
:104600001C91003050E0150781E009F080E09F9197
:10461000892B882311F40C94CF22C49AA881B981E4
:104620000D911C91003050E0150711F00C942023DF
:10463000ECE1F0E60E94D82D0E94E42D0C947B253D
:10464000A89584E690E00E94912EA895C49881E0F8
:1046500090E00E94912EEE81FF81FA93EA935A92A4
:104660004A9280E5A42DB52D8C9381E00E942C2DDB
:104670005A924A9201E010E020E030E0A42DB52DDE
:104680000D931D932D933C9384E00E942C2D0E944A
:104690005E28269685E00E94282D85E090E00E9405
:1046A000912EC49A8AE090E00E94912EA89500E095
:1046B00010E020E030E0AAE7B0E00D931D932D93C9
:1046C0003C9300E010E020E030E0A3EDB0E00D937B
:1046D0001D932D933C930E94812500E010E020E083
:1046E00030E0A3EDB0E00D931D932D933C93002794
:1046F000A1EDB0E08C9186FB0EF401E041E00417DF
:1047000011F00C9485230C947B25A8950091E8006A
:10471000023011F40C94192480919E0280937E0043
:10472000A5EAB2E00D91112740E051E00E94AB2DC7
:10473000AA81BB810D931C93AA81BB810D911C9111
:10474000A4EAB2E04D915527040F151FAA81BB8141
:104750000D931C93AA81BB810D911C9122273327B5
:1047600040E050E061E070E00E94F12DAAE7B0E087
:104770000D931D932D933D93A3EAB2E00D91112764
:1047800040E051E00E94AB2DAA81BB810D931C93A8
:10479000AA81BB810D911C91A2EAB2E04D915527EF
:1047A000040F151FAA81BB810D931C93AAE7B0E0EB
:1047B0000D911D912D913C91AA81BB814D915C91F0
:1047C000662777270E94F82EAAE7B0E00D931D9385
:1047D0002D933D9300917E000C3011F00C94F32347
:1047E0008BE080937E0000917E000E3011F00C94DF
:1047F000FC238BE080937E0000917E000F3011F04F
:104800000C9405248BE080937E00AAE7B0E00D9124
:104810001D912D913C91A3EDB0E00D931D932D932F
:104820003C930E948125A3EDB0E00E944B2D0C9497
:104830006D2400911201063411F00C94432484E09D
:1048400080937E0087E3A885B9858C93A885B98578
:104850000C910C3318F011F00C944124A885B98503
:10486000AD90BB24ABEDB0E0AA0DBB1D8C910E94B6
:10487000E72DA885B9858C918F5F8C9311F00C94EE
:1048800026240E94E42D00912E01063411F00C9490
:104890006D248BE080937E0083E5A885B9858C9399
:1048A000A885B9850C91073518F011F00C946B248C
:1048B000A885B985AD90BB24ABEDB0E0AA0DBB1DBA
:1048C0008C910E94E72DA885B9858C918F5F8C9380
:1048D00011F00C9450240E94E42DE6E2F0E60E94D0
:1048E000D82DA8E6B7E0EEE7F0E00E94242F0E9462
:1048F000D02D0E94E42DE8E3F0E60E94D82DA8E632
:10490000B7E0EAE7F0E00E94182F0E94D02D0E9445
:10491000E42D84E0A885B9858C93A885B9850C9190
:104920000B3018F011F00C94A824A885B985AD902F
:10493000BB24ABEDB0E0AA0DBB1D8C910E94E72D0E
:10494000A885B9858C918F5F8C9311F00C948D2480
:104950000E94E42D8091E90080936F00EAE4F0E684
:104960000E94D82DA8E6B7E0EFE6F0E00E94242FE1
:104970000E94D02D0E94E42D00916F00003011F0B4
:104980000C94C4240C947B2500916F00003418F023
:1049900011F00C94CD240C94CF240C947B258091A1
:1049A000EA00AE81BF818C938091EB00AC81BD8128
:1049B0008C93AC81BD819C91AE81BF818C91ADE621
:1049C000B0E08D939C938091F200AE81BF818C9377
:1049D0008091F300AC81BD818C93AC81BD819C91B1
:1049E000AE81BF818C91A0E7B0E08D939C93A0E74E
:1049F000B0E00D911C91003050E0150711F00C94BF
:104A0000172580910001AE81BF818C9380910101B7
:104A1000AC81BD818C93AC81BD819C91AE81BF8105
:104A20008C91A0E7B0E08D939C930C941725A0E7A0
:104A3000B0E00D911C91003050E0150711F00C947E
:104A400023250C947B2502E010E020E030E0A0E775
:104A5000B0E04D915C91662777270E94F12DA2E787
:104A6000B0E00D931D932D933D93A2E7B0E00D911F
:104A70001D912D913C91ADE6B0E04D915C91662782
:104A800077270E94F82EA2E7B0E00D931D932D9397
:104A90003D93A2E7B0E00D911D912D913C91A3EDC6
:104AA000B0E04D915D916D917C910E94F82EA2E74E
:104AB000B0E00D931D932D933D93EAE5F0E60E943F
:104AC000D82DA8E6B7E0E2E7F0E00E94182F0E9498
:104AD000D02D0E94E42DA2E7B0E00D911D912D9103
:104AE0003C91A3EDB0E00D931D932D933C9380E09A
:104AF000AA85BB858C9387E0481A8827580A2A968E
:104B0000089581E00E94A02E81E00E94A02E82E004
:104B10000E94A02E82E00E94A02E8FEFAE81BF8166
:104B20008C9391E0AE81BF810E94732E91E0AE81A3
:104B3000BF810E94732E91E0AE81BF810E94732ECF
:104B400091E0AE81BF810E94732E91E0AE81BF8162
:104B50000E94732E91E0AE81BF810E94732E91E07E
:104B6000AE81BF810E94732E91E0AE81BF810E9411
:104B7000732E91E0AE81BF810E94732E91E0AE81D1
:104B8000BF810E94732E91E0AE81BF810E94732E7F
:104B900091E0AE81BF810E94732E91E0AE81BF8112
:104BA0000E94732E91E0AE81BF810E94732E91E02E
:104BB000AE81BF810E94732E91E0AE81BF810E94C1
:104BC000732EC49880E090E0A881B9818D939C9366
:104BD0008FEF0E94842E0E94862E0E94852EAE8129
:104BE000BF818C93A881B9810E943F2DAE81BF8186
:104BF0000C91003081E009F480E08F93A881B981A5
:104C00000D911C91003050E0150781E009F080E023
:104C10009F91892B882311F40C94E825A881B981F0
:104C20000D911C91003050E0150711F00C942526D1
:104C3000E2E6F0E60E94D82D0E94E42D7091D100AA
:104C400070647093D1000C947227EE81FF81FA9307
:104C5000EA935A924A9281E5A42DB52D8C9381E076
:104C60000E942C2D5A924A92A3EDB0E00D911D9115
:104C70002D913C91A42DB52D0D931D932D933C9317
:104C800084E00E942C2D0E945E28269685E00E94DA
:104C9000282D0027A1EDB0E08C9186FB0EF401E0F9
:104CA00041E0041711F00C946526E0E7F0E60E945D
:104CB000D82DA8E6B7E0E3EDF0E00E94182F0E949F
:104CC000D02D0E94E42D0C947227A895AE81BF814F
:104CD0000C91003011F00C94B02680E090E0A88197
:104CE000B9818D939C938FEF0E94842E0E94862E13
:104CF0000E94852EAE81BF818C93A881B9810E94CC
:104D00003F2DAE81BF810C91003081E009F480E03D
:104D10008F93A881B9810D911C91003050E0150747
:104D200081E009F080E09F91892B882311F40C9495
:104D30007326A881B9810D911C91003050E01507B0
:104D400011F00C94B026EAE8F0E60E94D82D0E94FB
:104D5000E42D7091D10070647093D1000C9472278F
:104D6000AE81BF810C910F3F11F00C94FA2680E0C8
:104D700090E0A881B9818D939C938FEF0E94842E3F
:104D80000E94862E0E94852EAE81BF818C93A881C1
:104D9000B9810E943F2DAE81BF810C910F3F81E010
:104DA00009F480E08F93A881B9810D911C910030A6
:104DB00050E0150781E009F080E09F91892B88235E
:104DC00011F40C94BD26A881B9810D911C9100307D
:104DD00050E0150711F00C94FA26E8E9F0E60E947D
:104DE000D82D0E94E42D7091D10070647093D10091
:104DF0000C947227AE81BF810C910E3F11F40C947C
:104E00001727E6EAF0E60E94D82DA8E6B7E0EE8183
:104E1000FF810E94242F0E94D02D0E94E42DC49A6D
:104E20007091D10070647093D1000C94722780E06F
:104E300090E0AA81BB818D939C9380E0AE81BF817D
:104E40008C93AE81BF810C910F3F18F011F00C9440
:104E50005927AA81BB810E943F2D8FEF0E94842E8B
:104E60000E94862E0E94852EAA81BB81AD90BC90A7
:104E7000ABEDB0E0AA0DBB1D8C93AA81BB810E9453
:104E80003F2D8FEF0E94842E0E94862E0E94852E39
:104E9000AA81BB81AD90BC90ABEDB0E0AA0DBB1D6B
:104EA0008C93AE81BF818C918F5F8C9311F00C94A9
:104EB00021278FEF0E94842E0E94862E0E94852E2D
:104EC000AE81BF818C938FEF0E94842E0E94862E2C
:104ED0000E94852EAE81BF818C93C49AA3EDB0E071
:104EE0000E94302D86E0481A8827580A289608958F
:104EF00082E00E94A02E81E00E94A02E80E0AE8180
:104F0000BF818C930E942422C49880E090E0AA8103
:104F1000BB818D939C938FEF0E94842E0E94862EDE
:104F20000E94852EA881B9818C93AA81BB810E94A1
:104F30003F2DA881B9810C91003081E009F480E017
:104F40008F93AA81BB810D911C91003050E0150711
:104F500081E009F080E09F91892B882311F40C9463
:104F60008B27AA81BB810D911C91003050E0150761
:104F700011F00C94C827E2E6F0E60E94D82D0E94BA
:104F8000E42D7091D10070647093D1000C94582876
:104F9000E881F981FA93EA935A924A9281E5A42D25
:104FA000B52D8C9381E00E942C2D5A924A92AA85AD
:104FB000BB850D911D912D913C91A42DB52D0D9387
:104FC0001D932D933C9384E00E942C2D0E945E281B
:104FD000269685E00E94282DA881B9810C91003089
:104FE00011F00C941F2880E090E0AA81BB818D9382
:104FF0009C938FEF0E94842E0E94862E0E94852E05
:10500000A881B9818C93AA81BB810E943F2DA88180
:10501000B9810C91003081E009F480E08F93AA817E
:10502000BB810D911C91003050E0150781E009F023
:1050300080E09F91892B882311F40C94F927A88193
:10504000B9810C910F3F11F00C94522880E090E050
:10505000AA81BB818D939C938FEF0E94842E0E9426
:10506000862E0E94852EA881B9818C93AA81BB814E
:105070000E943F2DA881B9810C910F3F81E009F476
:1050800080E08F93AA81BB810D911C91003050E08C
:10509000150781E009F080E09F91892B882311F4A6
:1050A0000C942C28A881B9818C91AE81BF818C93FE
:1050B00083E0481A8827580A2496089584E00E94BD
:1050C000A02E81E00E94A02E82E00E94A02E8FEFF1
:1050D000AA81BB818C9391E0AA81BB810E94732E2F
:1050E00091E0A885B9850E94732EAE81BF810D9194
:1050F0001D912D913C9140E052E060E070E00E94F3
:10510000F12DAC81BD810D931D932D933D93AC8109
:10511000BD818F9314968E910E94E4288E910E94F7
:10512000E4288E910E94E4288E910E94E42885E96B
:105130000E94E4288F9180E090E0A881B9818D934E
:105140009C938FEF0E94842E0E94862E0E94852EB3
:10515000AA81BB818C93A881B9810E943F2DAA812D
:10516000BB810C910F3F81E009F480E08F93A8810F
:10517000B9810D911C91003050E0150781E009F0D4
:1051800080E09F91892B882311F40C94A128A88199
:10519000B9810D911C91003050E0150711F00C946D
:1051A000DC28E4EBF0E60E94D82D0E94E42D7091FB
:1051B000D10070647093D100AA81BB818C91AA85C3
:1051C000BB858C930C94E9288FB9779BFECF8FB168
:1051D000089587E0481A8827580A269608955A9213
:1051E0004A9284E298E0A42DB52D8D939C9382E0A1
:1051F0000E942C2D5A924A9280E0A42DB52D8C93BA
:1052000081E00E942C2D0E94D72B249683E00E94DF
:10521000282DEF93FF93ECE8F1E00E94652EFF91BB
:10522000EF91BB27A0E38C9182FBDEF789E190E050
:105230000E94912E5A924A9280E298E0A42DB52DB8
:105240008D939C9382E00E942C2D5A924A9280E08A
:10525000A42DB52D8C9381E00E942C2D0E94D72B7C
:10526000249683E00E94282D89E190E00E94912EEF
:105270000E945F2A089582E00E94A02E82E00E9490
:10528000A02E82E00E94A02EA885B9850C91003046
:1052900081E009F080E08F93AE81BF810C910030F6
:1052A00081E009F080E09F918923882311F40C9418
:1052B0006B29AA85BB858C91AA81BB818D93882798
:1052C0008C93AA85BB858C91A881B9818D93882701
:1052D0008C930C94AD29AA85BB850D911127A885C7
:1052E000B9854D915527040F151FAA81BB810D93D8
:1052F0001C93AA81BB810D911C910F3F50E01507B3
:1053000018F011F00C9486290C948C298FEF90E002
:10531000AA81BB818D939C93AA85BB850D91112792
:10532000AE81BF814D915527040F151FA881B9810A
:105330000D931C93A881B9810D911C910F3F50E0F2
:10534000150718F011F00C94A7290C94AD298FEFD4
:1053500090E0A881B9818D939C9300E011E0AA812F
:10536000BB814D915C910E94AB2DAC81BD810D93B1
:105370001C93AC81BD810D911C91A881B9814D9187
:105380005C91040F151FAC81BD810D931C935A9243
:105390004A92AE81BF818D919C91A42DB52D8D93A4
:1053A0009C9382E00E942C2D5A924A928BE0A42D6D
:1053B000B52D8C9381E00E942C2D0E94D72B249632
:1053C00083E00E94282D5A924A9280E298E0A42D10
:1053D000B52D8D939C9382E00E942C2D5A924A9277
:1053E00080E0A42DB52D8C9381E00E942C2D0E948D
:1053F000D72B249683E00E94282D86E0481A882720
:10540000580A2696089582E00E94A02E00E110E03E
:10541000AC81BD814D9155270E94AB2DA881B981EA
:105420000D931C93A881B9810D911C91AA81BB8118
:105430004D915527040F151FA881B9810D931C9319
:105440005A924A92AA81BB818D919C91A42DB52D2F
:105450008D939C9382E00E942C2D5A924A9282E076
:10546000A42DB52D8C9381E00E942C2D0E94D72B6A
:10547000249683E00E94282D82E0481A8827580A43
:10548000229608955A924A92AA81BB818D919C914D
:10549000A42DB52D8D939C9382E00E942C2D5A92C1
:1054A0004A9283E0A42DB52D8C9381E00E942C2D8F
:1054B0000E94D72B249683E00E94282D089581E036
:1054C0000E94A02E81E00E94A02EC49AD898C29873
:1054D00080E0A881B9818C9380E0AA81BB818C9304
:1054E000AA81BB810C910F3118F011F00C94942A11
:1054F00091E0A881B9810E94732E91E0A881B981C1
:105500000E94732E91E0A881B9810E94732E91E0D0
:10551000A881B9810E94732EAA81BB818C918F5F73
:105520008C9311F00C94702AC29AD89A82E0481A8F
:105530008827580A2496089581E00E94A02E5A9246
:105540004A9280E298E0A42DB52D8D939C9382E041
:105550000E942C2D5A924A9280E0A42DB52D8C9356
:1055600081E00E942C2D0E94D72B249683E00E947C
:10557000282DAA81BB810C91003011F00C94CF2A08
:105580005A924A9280E0A42DB52D8C9381E00E941E
:105590002C2D0E94492B229681E00E94282DAA8161
:1055A000BB810C91013011F00C94E52A5A924A9279
:1055B00085E6A42DB52D8C9381E00E942C2D0E94B0
:1055C000492B229681E00E94282DAA81BB810C9153
:1055D000023011F00C94122B5A924A9283E6A42DB9
:1055E000B52D8C9381E00E942C2D0E94492B229690
:1055F00081E00E94282D88EC90E00E94912E5A9222
:105600004A9280E0A42DB52D8C9381E00E942C2D30
:105610000E94492B229681E00E94282D82E390E08F
:105620000E94912EAA81BB810C91033011F00C9441
:105630003B2B5A924A9282E6A42DB52D8C9381E0A1
:105640000E942C2D0E94492B229681E00E94282D39
:1056500080E991E00E94912E5A924A9280E0A42D16
:10566000B52D8C9381E00E942C2D0E94492B22960F
:1056700081E00E94282D8AE090E00E94912E8AE02D
:1056800090E00E94912E81E0481A8827580A2296BD
:10569000089581E00E94A02EC49AD898C298AA8149
:1056A000BB810C91003018F011F00C94592B0C9424
:1056B000932B83E5A881B9818C9391E0A881B9816E
:1056C0000E94732E8FEEA881B9818C9391E0A881FE
:1056D000B9810E94732E8EE6A881B9818C9391E0E6
:1056E000A881B9810E94732E91E0AA81BB810E949A
:1056F000732E80E0A881B9818C9391E0A881B98153
:105700000E94732E91E0A881B9810E94732E91E0CE
:10571000A881B9810E94732E91E0A881B9810E946D
:10572000732E0C94CF2B85E4A881B9818C9391E0E2
:10573000A881B9810E94732E88E7A881B9818C93D2
:1057400091E0A881B9810E94732E89E6A881B98170
:105750008C9391E0A881B9810E94732E84E7A8817F
:10576000B9818C9391E0A881B9810E94732E80E069
:10577000A881B9818C9391E0A881B9810E94732E90
:1057800091E0A881B9810E94732E91E0A881B9812E
:105790000E94732E91E0A881B9810E94732EC29A53
:1057A000D89A81E0481A8827580A2296089581E0FD
:1057B0000E94A02EC29AD8985A924A9282E0A42DB2
:1057C000B52D8C9381E00E942C2D0E948C2C22966A
:1057D00081E00E94282D5A924A92AC81BD818C9121
:1057E000A42DB52D8C9381E00E942C2D0E948C2C31
:1057F000229681E00E94282DAC81BD8111968C916A
:10580000A881B9818C935A924A92AA81BB818C91CA
:10581000A42DB52D8C9381E00E942C2D0E948C2C00
:10582000229681E00E94282DAC81BD818C91A881B7
:10583000B9818C935A924A92AA81BB818C91A42DF2
:10584000B52D8C9381E00E942C2D0E948C2C2296E9
:1058500081E00E94282DD89A81E0481A8827580AAA
:105860002296089581E00E94A02E81E00E94A02E41
:1058700082E00E94A02EC29AD8985A924A9283E05F
:10588000A42DB52D8C9381E00E942C2D0E948C2C90
:10589000229681E00E94282D5A924A92A885B985C5
:1058A0008C91A42DB52D8C9381E00E942C2D0E940B
:1058B0008C2C229681E00E94282DEC81FD81FA93A8
:1058C000EA930E94922C2296EA81FB81FA93EA9352
:1058D0000E94922C2296D89AAC81BD810D911127FD
:1058E00040E051E00E94AB2DA881B9810D931C933B
:1058F000A881B9810D911C91AA81BB814D91552739
:10590000040F151FA885B9850D931C9384E0481AD0
:105910008827580A2696089591E0A881B9810E94A7
:10592000732E089581E00E94A02E91E0A881B98194
:105930000E94682EA881B9818C91AA81BB818C9329
:1059400081E0481A8827580A2296089582E00E942A
:10595000A02E81E00E94A02EC49ABB27A0E38C91C8
:1059600082FBDEF7C298AC81BD810D911C910030A5
:1059700052E0150711F00C94F52C81E090E0AA811B
:10598000BB818D939C9380E0A881B9818C93A88181
:10599000B9810C910F3018F011F00C94F32CBB2747
:1059A000A0E38C9182FBDEF790E2AA81BB81AD90EF
:1059B000BC90ABEDB0E0AA0DBB1D0E94732EAA8176
:1059C000BB810D911C9140E250E0040F151FAA818C
:1059D000BB810D931C93A881B9818C918F5F8C93AF
:1059E00011F00C94C72C0C94212D81E090E0AA8139
:1059F000BB818D939C93AC81BD814D915C91AA81BB
:105A0000BB810D911C910417150718F011F00C942F
:105A1000212DBB27A0E38C9182FBDEF7C29A91E097
:105A2000AA81BB81AD90BC90ABEDB0E0AA0DBB1DCF
:105A30000E94732EAA81BB810E943F2D11F00C940D
:105A4000FB2CC29A83E0481A8827580A24960895A6
:105A5000481A8827580A0895480E8827581E08951E
:105A60000D911D912D913C9181E0080F8827181F01
:105A7000281F381F3C932E931E930E930895ED918B
:105A8000FC913196FC93EE930895ED91FC91319742
:105A9000FC93EE9308950D911D912D913C91015031
:105AA0001040204030403C932E931E930E93089557
:105AB0004091DD025091DE020DE815E30E946C2D4D
:105AC00049E156E3040F151F0093DD021093DE0237
:105AD000498158810C94912D08D03DD000FC10D004
:105AE000089503D01ED001F8F9CF0024E89457FFA1
:105AF00002C009D0689400F80BD010F80124089572
:105B000002D009D00895509540954F5F5F4F08959A
:105B1000E89417FF0895009510950F5F1F4F689444
:105B20000895352F242FE894452B11F46894089597
:105B3000512F402F0027112780E1440F551F001FD0
:105B4000111F021B130B416018F4020F131F4E7F2D
:105B50008A9599F708950F92049F202C312C419F2C
:105B6000300C509F030C022D102D0F900895C895F6
:105B70000D9231960020D9F708958F938D91882347
:105B8000E9F711978F91089581E05F9B8827089529
:105B900088275F9B089500C05F9BFECF8CB108955E
:105BA000A8E6B7E08D91882311F011D0FBCF0895BE
:105BB0000E94A62E802D11F00AD0FACF08958D9163
:105BC00006D03A95E1F708958DE001D08AE05D9B1B
:105BD000FECF8CB9089588EE93E0A3D03197D9F722
:105BE000089550D00AD000FC05D008954BD020D0A5
:105BF00001F8F9CF52D05AD00895842F952FA62FAF
:105C0000B72F4427552766277727F1E2889409C0E4
:105C100020F4480F591F6A1F7B1F7695679557958B
:105C200047953795279517950795FA9589F708951C
:105C3000842F952FA62FB72FE894452B462B472B63
:105C400011F468940895402F512F622F732F00276D
:105C5000112722273327F0E2440F551F661F771FB5
:105C6000001F111F221F331F081B190B2A0B3B0B90
:105C7000416028F4080F191F2A1F3B1F4E7FFA9519
:105C800059F708950024E89477FF02C006D068947D
:105C900000F809D010F80124089512D04F5F5F4F2B
:105CA0006F4F7F4F0895E89437FF08950095109542
:105CB000209530950F5F1F4F2F4F3F4F68940895E9
:105CC000409550956095709508953197F1F7089536
:105CD0000E94842E8C910E94862E8D939A95D1F7E6
:105CE0000E94852E08950E94842E8D910E94862EFA
:105CF0009A95D9F70E94852E0895BF9ABE98C69AA4
:105D0000BD9A80E58DB90895089508958FB9779B60
:105D1000FECF8FB10895689462F80895E89462F810
:105D20000895EF93FF93EE27E82BE92B31F0E0ED98
:105D3000F7E03197F1F70197D1F7FF91EF910895CF
:105D40005A924A92480E8827581E0895C89531964F
:105D500000200895819104D08D938823D9F7089568
:105D6000813618F08B3708F48F7D089580E30EF4A8
:105D7000839508952E2E3F2E992781918D3209F01B
:105D800093958823D1F79A95E22DF32D112361F095
:105D9000091718F011F0101B01C0191B28F021F091
:105DA00080E28D931A95E9F780818D3219F48D93F5
:105DB000319604C0222311F08BE28D93091738F03D
:105DC00031F0091B21F080E38D930A95E9F7819169
:105DD0008D938823E1F7332351F0EA2FFB2F31967F
:105DE00033958E9182933A95E1F78EE28C930895E4
:105DF000040F151F261F371F0895041B150B260BB4
:105E0000370B089504171507260737070895000F65
:105E1000111F221F331F089500951095209530956E
:105E20000F5F1F4F2F4F3F4F0895019110810EC0FC
:105E300001911191219130810BC00191108117FFC7
:105E400005C03FEF2FEF04C0008111272227332721
:105E500037FF03C0E1DF8DE28D93CF93DF93CF92C5
:105E6000DF92EF92AA24BB24CC24DD24EE2440E26E
:105E7000CAE0DD2755E093E38881890F87FD9F7095
:105E800083FD907F891B89935A95A9F7C0DFAA1CCF
:105E9000BB1CCC1CDD1CEE1C4A9551F7E894EFE0CE
:105EA000FF2782910ED0EB30E0F71EF068948A2D28
:105EB0000CD088278D93EF90DF90CF90DF91CF911A
:105EC0000895982F829501D0892F8F70805D26F0DC
:105ED000803309F4089568948D93089588278D93ED
:105EE000089581918D938823E1F708950991919107
:105EF000992351F08A95D9F7319781918D930A951D
:105F000019F08823D1F70895E9CFE199FECFEEBBD0
:105F1000FFBB3196089591E001C092E07B3751F4C8
:105F20007FB7F894F2DF8D918DBBE29AE19A9A9552
:105F3000C9F77FBF7727089591E001C092E0E5DFC0
:105F4000E09A8DB38D939A95D1F70895FF93881BAE
:105F5000F9E0001FFA9511F4FF910895881F841B42
:105F600018F4840F8894F5CF0894F3CF689401C097
:105F7000E894AF93BF938D9116F0919103C00E9466
:105F8000A62E902D891718F011F48823A1F7BF9140
:105F9000AF9108954D50335354414D502052656197
:105FA0006C6974792D53797320342E3600005300B8
:105FB0005000454570726F6D20002C004D4D432000
:105FC000696E697420007265747279202E2E2E001D
:105FD00044535020696E697420004F005A005900E4
:105FE0004700520057004100480021004E00420087
:105FF00058004400450056004D00540049004C0034
:10600000434F4E46494700002000442000002E0028
:106010006F6B00004E6F2063617264004261642008
:10602000636172640000506172746974696F6E20FC
:1060300074797065203A0000506172746974696FF8
:106040006E2073746172743A0000536563742F6339
:106050006C757374657220203A00526F6F74203A29
:10606000000052656164206572726F722031000019
:1060700052656164206572726F722032206F6E20EB
:10608000736563746F723A20000052656164206525
:1060900072726F7220330000526561642065727203
:1060A0006F722034000052656164206572726F72F5
:1060B00020350000526561642074696D656F7574E8
:0260C0000000DE
:00000001FF
